:10000000342883169B001C141A082F2883169A0084
:100010001C1555309D00AA309D009C149C180E287C
:100020001C112F28A301A200FF30A207031CA30765
:10003000031C2F280330A100E63020201428A10142
:10004000FC3EA000A109031C2B28FF300000A007E4
:1000500003182628A0076400A10F25280800831391
:10006000031383126400080025309F008316F130CB
:100070009F00051085158516051683120330A30011
:10008000E830132000300120B80064001530380239
:10009000031C4C281430B8006400013038020318E7
:1000A00053280130B8006400851D60286400851E57
:1000B0007C286400051E982864009F1BB3285328E1
:1000C000B80A640015303802031C68281430B800E0
:1000D000831605128312051283160512C830831287
:1000E000122005168316051283126400851D7528DB
:1000F0008316051683125328B803640001303802B2
:10010000031884280130B8008316051283120512E3
:1001100083160512C83083121220051683160512A5
:1001200083126400851E91288316051683125328B6
:10013000C0200330A300E830132083169B018312F4
:10014000380806208316051283120512831605123D
:1001500083120330A300E83013200516831605121E
:1001600005168312532805108316051083123808CC
:1001700012200514831605106430831212205328B0
:100180000330A300E83013200130B90064003908BF
:100190003802031CDE28831605128312051283160B
:1001A000051264308312122005168316051283127D
:1001B0000130A3002C301320B90FC6288316051672
:0A01C0008312080053286300E328AF
:02400E00623F0F
:00000001FF
